:100000000C941E060C94B0260C94DD260C94460627
:100010000C9446060C9446060C9446060C94460630
:100020000C9446060C9446060C9405120C94460655
:100030000C9446060C9446060C9446060C94460610
:100040000C940A270C9446060C94F82A0C943B2B2B
:100050000C9446060C9446060C9446060C944606F0
:100060000C9446060C9446066117C317A217A517F1
:10007000A817AB17AE17B117B417C317BD17F518EC
:10008000F718F718F518F718F718F718F718F718FA
:10009000F718F718F718F718F718F718F718F718E8
:1000A0007B18F718F718F718F718F718EC17F71860
:1000B000F718F718F718F718F718F718F718F718C8
:1000C000F718F718F718F718F718F7188718871898
:1000D0008718871887188718871887188718F718B8
:1000E000F718F718F718F718F718EC178618861886
:1000F00086188618F71894189A18A018A618AC181D
:10010000B218B818BE18C818D218DC18E6182D187E
:10011000EF17F718F718F718F7187B18F718F718EC
:10012000F718F718F718F718F718F718851885183B
:1001300085188518F71894189A18A018A618AC18DE
:10014000B218B818BE18C818D218DC18E6182D183E
:10015000EF17F718F718F718F7187B182A192A1944
:100160002A192A192A192A192A192A192A192A1977
:100170002A192A192A19411A411A411A411A411AEF
:10018000411A6F19791983198D19EB19F519041A88
:10019000151A9C1BB11BBD1BC61BD51BFA1B031CD0
:1001A0004C1C151C431F491F4F1F561F641F861FE1
:1001B000A41F456E746572206D656E752E2E2E001F
:1001C000546F67676C6564206D6963726F50504D42
:1001D00000546F67676C656420696E76657274653C
:1001E000642050504D2100546F67676C6564205443
:1001F00058206D7574696E672100546F67676C6570
:10020000642074656C656D65747279210050726F3D
:10021000746F636F6C206572726F72207769746897
:100220002052580054696D656F7574207768656E4B
:1002300020636F6E6E656374696E6720746F205201
:100240005800507265737320616E79206B65792058
:10025000746F2063616E63656C00436F6E6E6563DF
:1002600074696E6720746F2052582C20706F776508
:100270007220757020746865205258202877697440
:10028000682062696E6420706C7567206966206EF4
:100290006F74207573696E6720616C776179732064
:1002A00062696E642900546F67676C656420276912
:1002B0006D6D656469617465206F75747075742700
:1002C00000546F67676C65642027736C61766520E6
:1002D0006D6F64652700546F67676C6564202761E4
:1002E0006C776179732062696E642700546F676769
:1002F0006C65642050504D206368616E6E656C20A3
:100300006C696D69740053657420525353492069B8
:100310006E6A656374696F6E206368616E6E656C8A
:100320002028303D3D64697361626C652900536526
:10033000742050504D206D696E696D756D20737914
:100340006E630053657420626561636F6E20696E31
:1003500074657276616C0053657420626561636FC9
:100360006E2064656C617900536574206265616319
:100370006F6E206672657175656E637920696E2097
:10038000487A3A20303D64697361626C652C205074
:10039000783D504D52206368616E6E656C20782CFC
:1003A0002046783D465253206368616E6E656C202E
:1003B00078005365742050574D2073746F7020641B
:1003C000656C61792028302064697361626C6564B2
:1003D0002C20312D323535203D3D20302E317320FB
:1003E0002D2035306D696E29005365742050504DB5
:1003F0002073746F702064656C61792028302064EC
:10040000697361626C65642C20312D323535203D75
:100410003D20302E3173202D2035306D696E29003E
:10042000536574206661696C736166652064656CF0
:1004300061792028302064697361626C65642C20C6
:10044000312D323535203D3D20302E3173202D2089
:1004500035306D696E29002A2A2A2A2A2A2A2A2A50
:100460002A2A2A2A2A2A2A2A2A2A2A2A2A2A2A2AEC
:100470002A2A2A2A0052582041636B6564202D20C5
:1004800072657665727420737563636573736675E0
:100490006C21002A2A2A2A2A2A2A2A2A2A2A2A2AAD
:1004A0002A2A2A2A2A2A2A2A2A2A2A2A2A2A2A2AAC
:1004B000002A2A2A2A2A2A2A2A2A2A2A2A2A2A2AC6
:1004C0002A2A2A2A2A2A2A2A2A2A2A2A2A2A00528E
:1004D000582041636B6564202D20757064617465DC
:1004E000207375636365737366756C21002A2A2A0D
:1004F0002A2A2A2A2A2A2A2A2A2A2A2A2A2A2A2A5C
:100500002A2A2A2A2A2A2A2A2A2A0056616C696457
:100510002063686F69636573206172653A205B319F
:100520005D2D5B31365D20286368616E6E656C20E1
:10053000312D31362900536574206F7574707574D0
:1005400020666F7220706F727420005B585D2061AE
:10055000626F7274206368616E67657320616E6498
:10056000206578697420525820636F6E6669670051
:100570005B535D20736176652073657474696E6783
:100580007320746F205258005B525D20726576654F
:1005900072742052582073657474696E6773207486
:1005A0006F2064656661756C747300557365206EA9
:1005B000756D62657273205B312D445D20746F2010
:1005C0006564697420706F727473205B452D515D92
:1005D00020666F722073657474696E677300202DD6
:1005E00020726563656976657220636F6E66696700
:1005F000757261746F722C20727820737720000AF4
:100600000A6F70656E4C52536E67200053657420FC
:1006100073657269616C2062617564726174653AB8
:10062000200056616C69642063686F696365733A82
:100630002031202D20342B34202F2032202D203823
:10064000202F2033202D20382B34202F2034202D14
:10065000203132202F2035202D2031322B34202FF5
:100660002036202D20313600536574204368616E9A
:100670006E656C20636F6E6669673A20005365741F
:100680002044617461726174652028302D32293AEA
:10069000200053657420486F70206368616E6E653A
:1006A0006C7320286D61782032342C207365706162
:1006B000726174656420627920636F6D6D61732966
:1006C0002076616C69642076616C75657320312DCC
:1006D0003235353A2000536574206368616E6E656B
:1006E0006C2073706163696E6720287831306B48C5
:1006F0007A293A200053657420524620706F77653E
:10070000722028302D37293A200053657420524634
:10071000206D6167696320286865782920652E67E8
:100720002E20307844454144463030443A2000532E
:1007300065742062617365206672657175656E63AC
:10074000792028696E20487A293A20005B5A5D207A
:10075000656E746572207265636569766572206383
:100760006F6E66696775726174696F6E2075746902
:100770006C79005B465D20646973706C61792061FF
:10078000637475616C206672657175656E63696509
:10079000732075736564005B525D2063616C6375E3
:1007A0006C6174652072616E646F6D206B65792079
:1007B000616E6420686F70206C697374005B495DC2
:1007C000207265696E697469616C697A6520736508
:1007D0007474696E677320746F20736B65746368DB
:1007E0002064656661756C7473005B585D2072658A
:1007F00076657274206368616E67657320616E64EC
:100800002065786974206D656E75005B535D20739B
:100810006176652073657474696E677320746F20E8
:10082000454550524F4D20616E64206578697420B3
:100830006D656E7500557365206E756D62657273BA
:10084000205B302D395D20746F20656469742070E1
:100850006172616D657465727300202D2053797328
:1008600074656D20636F6E66696775726174696F18
:100870006E000A0A6F70656E4C52536E672000510D
:1008800029204F7574707574206265666F726520DB
:100890006C696E6B20283D465329203A2000502970
:1008A00020536C617665206D6F64652028657870D3
:1008B0006572696D656E74616C293A20004F29205C
:1008C00054696D65642042494E44206174207374FC
:1008D000617274757020203A20004E292050504DCE
:1008E000206F7574707574206C696D69746564200F
:1008F000202020203A200044495341424C454400E6
:100900004D292050504D205253534920746F20637D
:1009100068616E6E656C202020203A20004C2920F2
:1009200050504D206D696E696D756D2073796E63E1
:10093000202875732920203A200044495341424C15
:100940004544004B29204661696C736166652062ED
:100950006561636F6E20696E74762E2028312D32AA
:10096000353573293A20004A29204661696C736144
:10097000666520626561636F6E2064656C617920D5
:1009800028302D323535203D3E20313073202D204A
:100990003135306D696E293A200049292046616958
:1009A0006C7361666520626561636F6E206672714B
:1009B0002E203A200048292050574D2073746F7024
:1009C0002064656C6179202020202020203A2000BE
:1009D00047292050504D2073746F702064656C61FE
:1009E00079202020202020203A200046292046611E
:1009F000696C736166652064656C617920202020D4
:100A00002020203A200050574D206368616E6E65AB
:100A10006C200066756E6374696F6E3A2000292041
:100A2000706F72742000506F776572546F776572C3
:100A300000445446205548462033322D62697420C4
:100A400031306368004F70656E4C52536E67525878
:100A5000206D696E6920342F36636800466C7974A6
:100A6000726F6E2F4F72616E6765525820554846FF
:100A70002038636800525820747970653A20004429
:100A8000697361626C656400487A00203D3D200016
:100A900043616C63756C61746564207061636B6540
:100AA0007420696E74657276616C3A200042292068
:100AB0004D6963726F202868616C66292050504D23
:100AC000202020203A00412920496E766572746505
:100AD000642050504D20696E20202020203A0030A4
:100AE00029204D7574652062757A7A657220286DAB
:100AF0006F73746C79293A003929205365726961E2
:100B00006C2062617564726174653A00736D617224
:100B100074506F7274004672536B79005472616E38
:100B200073706172656E740044697361626C6564B0
:100B30000038292054656C656D657472793A2020FF
:100B40002020202020003729204368616E6E656CCC
:100B500020636F6E6669673A202000362920446161
:100B60007461726174652028302D32293A2020206A
:100B700000352920486F70206368616E6E656C7364
:100B80003A2020202020003429204368616E6E65C1
:100B90006C2073706163696E673A202000332920EE
:100BA000524620706F7765722028302D37293A2001
:100BB0002020003229205246206D616769633A2067
:100BC0002020202020202020003129204261736530
:100BD000206672657175656E63793A202020000089
:100BE00000000700020100000304060000000000EE
:100BF00000000001020408102040800102040810D7
:100C00002001020408102004040404040404040263
:100C10000202020202030303030303000000002395
:100C2000002600290000000000250028002B0000FD
:100C3000000000240027002A0000292C11241FBED8
:100C4000CFEFD8E0DEBFCDBF13E0A0E0B1E0E0E63B
:100C5000FEE502C005900D92AA39B107D9F716E05A
:100C6000AAE9B3E001C01D92AF35B107E1F71CE07E
:100C7000CCE3DCE004C02297FE010E94322DCA338F
:100C8000D107C9F70E94652C0C942E2F0C940000FC
:100C90008091A505813019F482E08093A5058091AB
:100CA000A505833019F484E08093A5050895A895DF
:100CB0000895DC01ED91FC910190F081E02D099502
:100CC000089582E08093B00085E08093B10061E0F8
:100CD00083E00E940D2860E083E00E94462808958A
:100CE0000097C9F09C0140E050E068E478EE81E0B4
:100CF00090E00E94DA2C2F3F31054105510529F083
:100D000020F02FEF30E040E050E02093B3008091DE
:100D1000B000806103C08091B0008F7E8093B000EE
:100D2000089560E08CE00E940D2861E08BE00E9455
:100D30000D2861E08DE00E940D2860E082E00E94B5
:100D40000D2861E084E00E940D28089542E050E003
:100D500068E476E080E00E9490260895E3E0F0E009
:100D600089E080935700E491E67081E0E63009F075
:100D700080E00895CF93DF93C82F0E94AE068823AA
:100D800081F0DFB781E08093A405F8940E945706B4
:100D900088E180936000C0936000C1110E945706F3
:100DA000DFBFDF91CF910895209144053091450533
:100DB000382748E0C901880F991F37FF06C09C01FA
:100DC00051E2252750E1352701C09C01415091F7A0
:100DD00030934505209344050895D82FC0E0CD17E2
:100DE00080F45E9A64E670E080E090E00E948327E1
:100DF0005E9864E670E080E090E00E948327CF5F19
:100E0000EECF6CE271E080E090E00E948327E6CFB5
:100E10000F931F93CF93DF93EC01062F15E0115032
:100E200051F0CE010E94152F081741F0602FCE011E
:100E30000E941D2FF4CF82E00E94ED06DF91CF913A
:100E40001F910F910895A0E0B0E0E9E2F7E00C9463
:100E5000FB2C482E562EC0E0D0E0612C712CE12CEA
:100E6000F12C00E010E041100CC06090A30586E476
:100E7000689E30011124A9E1EA2EF12C0AE815E060
:100E80001EC091E049120FC06090A305E6E46E9E7B
:100E900030011124FBE16F0E711CF9E2EF2EF12CF1
:100EA00006E415E00CC082E0481209C078E1672E24
:100EB00077247394EE24E394F12C03EA15E04301C4
:100EC0008C0E9D1E10924505109244053401A62CEF
:100ED000A818B12CC30101966C01AE14BF04A8F48C
:100EE000A00EB11E511006C0C3010E94152FF501BE
:100EF000808305C0F5016081C3010E940807F501E8
:100F000080810E94D4063601E2CFC301511018C07F
:100F1000C3010E94152FB82EC6010E94152F2B2D3C
:100F200030E0322F2227282B8091440590914505EF
:100F30008217930779F4C0E0D0E05524539493CFFF
:100F40003601609145050E94080760914405C6017D
:100F50000E940807C05EDE4FC13E92E0D90708F448
:100F600082CF852DCDB7DEB7E0E10C94172D87E356
:100F70008093460580E092ECA1E0B0E080934705C5
:100F800090934805A0934905B0934A0587E0809364
:100F9000530580EC92E9ADEEB9E180934B05909357
:100FA0004C05A0934D05B0934E0585E08093540504
:100FB0008DEE9EEFADEABEED80934F059093500508
:100FC000A0935105B0935205E5E5F5E080E090E08F
:100FD000863028F4DC01AC59BC4F2C9101C020E0D4
:100FE000219301968831910599F782E080936D05F0
:100FF0008AE080936E05089561E082E00E942307F5
:10100000089560E082E00E9423078091A305843068
:1010100020F01092A3050E94FC070895A1E0B0E023
:10102000E4E1F8E00C94092D89830E940108909175
:10103000A3058981981731F0843020F48093A305AB
:101040000E94FC072196E2E00C94252D80EC91EDA6
:10105000A8E9BBE180938B0590938C05A0938D0547
:10106000B0938E0580E090E0A0E0B0E580938F051E
:1010700090939005A0939105B0939205E3E9F5E074
:1010800080E081938F5F8031E1F70895A0E0B0E0C8
:10109000ECE4F8E00C94FF2C0E94602761157105C8
:1010A00081059105C9F30E949E2D10924F05109263
:1010B00050051092510510925205C4E0C12CD12C5C
:1010C0007601CA9480904F0590905005A0905105EC
:1010D000B0905205BA2CA92C982C88240E94992DE6
:1010E000A70196010E94DA2C680D791D8A1D9B1DAF
:1010F00060934F057093500580935105909352056E
:10110000C15001F705E515E0E801C12CD12CB2E38F
:101110008B2E912CA12CB12C80E1E82E87E2F82EA9
:101120008881882309F446C0D39419F40E94B70734
:1011300041C00E94992DA50194010E94DA2C21E062
:10114000260FE5E5F5E08E2F801B8C1520F48191AC
:101150008213F9CFE9CF40915405249FA0011124B7
:101160004E9DC0014F9D900D5E9D900D1124AA27AC
:1011700097FDA095BA2F40914B0550914C05609179
:101180004D0570914E05840F951FA61FB71F409106
:101190008B0550918C0560918D0570918E054817D7
:1011A00059076A077B0708F4BFCF2993C39488E1E6
:1011B000C812B6CFCDB7DEB7ECE00C941B2D61E0C2
:1011C00080E00E94230761E081E00E9423070895E8
:1011D00060E080E00E942307882331F060E081E036
:1011E0000E942307811108C00E9426080E94B707A9
:1011F0000E9446080E94DF0808958436910520F475
:10120000BC0180E090E017C09C018E3B910528F462
:101210002A553109AAE0B0E00CC0823D910528F4BE
:10122000245B3109A4E6B0E004C02D5C3109A8E5D7
:10123000B2E00E94722CA4E6B0E09B01AC010E94D7
:10124000812C089590E08C599F4F0E94FD080895CD
:101250008F929F92AF92BF92CF92DF92EF92FF92C6
:10126000CF93FC01C0A5EC2FE770F0E0E45BFC4FEE
:10127000A081B0E0C7FF03C024E130E002C02FE04E
:1012800030E0FC0197A183E1989FF0011124E25C1A
:10129000FE4F80809180A280B380A20FB31F20E414
:1012A0003FE14DE750E00E948C2CA50194010E9483
:1012B000B82C8C2F887149F469017A01E0EDCE0ECB
:1012C000E7E0DE1EE11CF11C1BC0C7FF05C060E4A7
:1012D0007AE88CE29EE004C060E07EEE8AEB9BE060
:1012E00069017A01F8EBCF0EFBE0DF1EE11CF11C77
:1012F000A50194010E94B82CC20ED31EE41EF51E57
:10130000C701B60169517C4F8F4F9F4F28EE33E0E4
:1013100040E050E00E94B82CA8EEB3E00E94812C7F
:10132000CF91FF90EF90DF90CF90BF90AF909F90C4
:101330008F9008958F3F910551F048F0811522E07C
:10134000920738F08115934030F482E0089580E0F0
:10135000089581E0089583E00895A0E0B0E0E3EB14
:10136000F9E00C94042DEB018A01B82FB695A0E0AA
:1013700028813981F80120832A813B8121832C81B6
:101380003D8122832E813F812383688179814A8137
:101390005B812C813D81EE81FF819F2F9295990F7A
:1013A000990F907C272F2370922B252F2370220FCB
:1013B000220F922B232F23702295207F922BF8014E
:1013C00094830B5F1F4F2896AF5FBA1788F680FF94
:1013D00024C0888199810E949A09D82E8A819B8194
:1013E0000E949A09E82E8C819D810E949A09F82E0C
:1013F0008E819F810E949A09F0E4DF9EA001112452
:1014000090E1E99E90011124242B282BE4E0FE9E1C
:10141000B0011124262BF8012083CDB7DEB7E7E019
:101420000C94202D803223E0920708F1883E23E0BF
:10143000920740F48F519340E4E096958795EA95A2
:10144000E1F70895803D27E0920718F48C5D934002
:101450000895883928E0920768F4885C974074E022
:10146000969587957A95E1F78D509C4F089580E089
:1014700090E008958FEF93E008958C30910540F44B
:10148000A4E0880F991FAA95E1F7885D9C4F089505
:10149000843F23E0920718F484529C4F08958115ED
:1014A00024E0920740F48657934FF4E0880F991F89
:1014B000FA95E1F7089580E998E008959C01369542
:1014C000279525753575821B930B9C012373337308
:1014D000969587959695879583739373820F931F3F
:1014E0009C0154E0369527955A95E1F7280F391F4E
:1014F0002F703F7041E051E0249FC001259F900D67
:10150000349F900D1124892F08952D98882319F068
:1015100000002B9A02C000002B9800002D9A0000BA
:1015200008952D9A000083B12D9800008295817056
:101530000895CF93DF93D82F5C9A2D985C98C8E0DC
:101540008D2F80780E94850ADD0FC150C9F72D9834
:10155000DF91CF9108958F770E94990A0895CF93D4
:10156000DF93D82FC8E08D2F80780E94850ADD0F89
:10157000C150C9F72D98DF91CF910895CF93DF9394
:101580002D98C8E080E0D82FDD0F0E94910A8D0FC2
:10159000C150C9F7DF91CF9108950E94AB0A0E9414
:1015A000BE0A5C9A0895A1E0B0E0E9EDFAE00C947F
:1015B000092D806869830E94990A6981862F0E949B
:1015C000AF0A5C9A2196E2E00C94252DCF93C0914E
:1015D0004F05C827E82FF0E0EA5BFA4F678589E7F7
:1015E0000E94D30A6C2F8DE30E94D30A6C2F82E4F1
:1015F0000E94D30ACF91089586E20E94CD0A0895F1
:10160000CF93DF93EC016C818CE10E94D30A6D8152
:101610008DE10E94D30A6E818EE10E94D30A6F8110
:1016200080E20E94D30A688581E20E94D30A69851C
:1016300082E20E94D30A6A8583E20E94D30A6B8504
:1016400084E20E94D30A6C8585E20E94D30A6D85EC
:101650008AE20E94D30A6E858EE60E94D30A6F85C5
:101660008FE60E94D30A688980E70E94D30A6989BD
:1016700081E70E94D30A6A8982E70E94D30ADF9138
:10168000CF910895CF92DF92EF92FF92CF93DF93A5
:101690006B017C01C11488E3D8068CE9E8068CE173
:1016A000F80628F5C701B60120E836E948E950E018
:1016B0000E94B82CE901689760E879E687E69FEF19
:1016C0000E94942C6C0D7D1D8E1D9F1DF2E0660FF7
:1016D000771F881F991FFA95D1F721E732E040E084
:1016E00050E00E94B82CF22EE32E80E421C0C70106
:1016F000B60120E03DE241E351E00E94B82CE9014F
:10170000689760E073ED8EEC9EEF0E94942C6C0D58
:101710007D1D8E1D9F1D660F771F881F991F21E756
:1017200032E040E050E00E94B82CF22EE32E80E63A
:101730006C2F6F71680F85E70E94D30A6E2D86E7C4
:101740000E94D30A6F2D87E70E94D30ADF91CF91C1
:10175000FF90EF90DF90CF900895682F8DE60E9464
:10176000D30A08958F929F92AF92BF92CF92DF9249
:10177000EF92FF92CF93DF93D82F61E089E00E9430
:10178000462862E370E080E090E00E94832760E0FA
:1017900089E00E94462862E370E080E090E00E94C9
:1017A000832783E00E94CD0A8093430584E00E9452
:1017B000CD0A8093420560E086E00E94D30A61E092
:1017C00087E00E94D30A6FE789E00E94D30A65E0B0
:1017D0008AE00E94D30A65E18BE00E94D30A62E1AD
:1017E0008CE00E94D30A6DEF8DE00E94D30A60E086
:1017F0008EE00E94D30ADD2319F08BE291E008C04D
:1018000020916D0533E1239FC0011124825C9E4F1E
:101810000E94000B6CE880E30E94D30A6FE082E331
:101820000E94D30A62E483E30E94D30A80916E058A
:1018300087FF02C064E101C06AE084E30E94D30A2A
:101840006AE285E30E94D30A6DE286E30E94D30A2E
:1018500064ED87E30E94D30A60E088E30E94D30A24
:1018600060E089E30E94D30AD11109C0C0904F05FE
:10187000D0905005E0905105F090520507C0C5E8A2
:10188000CC2EC1ECDC2EED2CCEEDFC2ECAE38F2C41
:101890009924AA24BB24682D8C2F0E94D30A682D7A
:1018A00085E08C0F0E94D30AFE2CED2CDC2CCC247E
:1018B000CF5FCE3361F76FEF83E40E94D30A6FEFFF
:1018C00084E40E94D30A6FEF85E40E94D30A6FEF8D
:1018D00086E40E94D30ADD2311F066E002C0609125
:1018E00053058DE60E94D30A60E089E70E94D30A7F
:1018F000609154058AE70E94D30A60E083E70E9462
:10190000D30A60E084E70E94D30AD11109C0609134
:101910004B0570914C0580914D0590914E0504C08A
:1019200060EC72E98DEE99E10E94420BDF91CF915C
:10193000FF90EF90DF90CF90BF90AF909F908F90EF
:10194000089561E087E00E94D30A64E28EE70E9476
:10195000D30A63E088E00E94D30A60E088E00E9436
:10196000D30A65E087E00E94D30A62E085E00E9426
:10197000D30A83E00E94CD0A8093430584E00E944D
:10198000CD0A80934205089583E00E94CD0A80939A
:10199000430584E00E94CD0A8093420561E087E020
:1019A0000E94D30A6AE070E080E090E00E94832702
:1019B0000E94A10C00000895CF92DF92FF920F9336
:1019C0001F93CF93DF931F92CDB7DEB7082F162F4B
:1019D0008EE399830E94D30AF02EC02E9981D92ECE
:1019E0008C2D8F19811738F4F60161916F018FE703
:1019F0000E94D30AF5CF64E085E00E94D30A83E019
:101A00000E94CD0A8093430584E00E94CD0A809312
:101A100042050E94602760933E0570933F058093C6
:101A200040059093410569E087E00E94D30A81E078
:101A30008093A5050F90DF91CF911F910F91FF909B
:101A4000DF90CF9008950F931F930E94DC0C80913C
:101A5000A505813099F40E94602700913E05109100
:101A60003F052091400530914105601B710B820BB1
:101A7000930B603A76488140910548F38091A50523
:101A8000813031F46EE971E083EB95E00E944C29DE
:101A90001F910F9108950F931F938091A505823098
:101AA00021F41092A50581E020C08091A505813028
:101AB000D9F40E94602700913E0510913F052091C6
:101AC000400530914105601B710B820B930B613A0D
:101AD00076488140910540F061E087E00E94D30A9A
:101AE0001092A50582E001C080E01F910F9108953A
:101AF000CF93DF93EC014AE050E06D2F70E083EB71
:101B000095E00E941A2A6EE283EB95E00E941E295E
:101B1000BE0184E0769567958A95E1F76F70772727
:101B20004AE050E083EB95E00E941A2A6EE283EBD4
:101B300095E00E941E29BE016F7077274AE050E0B1
:101B400083EB95E00E941A2ADF91CF9108958823B4
:101B500019F06AEA71E002C06EEA71E083EB95E089
:101B60000E944C290895FF920F931F93CF93DF9308
:101B700069EC7BE083EB95E00E94F82840914B05EF
:101B800050914C0560914D0570914E052AE030E072
:101B900083EB95E00E94212A63EB7BE083EB95E0E9
:101BA0000E94F82840914F055091500560915105D1
:101BB0007091520520E130E083EB95E00E94212AEC
:101BC0006DE97BE083EB95E00E94F8284AE050E065
:101BD0006091530583EB95E00E94492A67E87BE01A
:101BE00083EB95E00E94F8284AE050E060915405AC
:101BF00083EB95E00E94492A61E77BE083EB95E067
:101C00000E94F828C5E5D5E0F12C8E018881882353
:101C1000A9F0FF2031F061EB71E083EB95E00E94C9
:101C20001B2921964AE050E0F801608183EB95E0A2
:101C30000E94122AF394F8E1FF12E7CF83EB95E0BC
:101C40000E9426296BE57BE083EB95E00E94F82853
:101C50004AE050E060916D0583EB95E00E94492ACF
:101C600066E47BE083EB95E00E94F828E0916E0546
:101C7000E770F0E0EE0FFF1FEC5AFC4F60817181BE
:101C800083EB95E00E944C2961E37BE083EB95E0D8
:101C90000E94F82880916E058871883069F028F4D8
:101CA000811113C068E27BE00CC0803141F08831C3
:101CB00061F46CE07BE005C06CE17BE002C066E1B2
:101CC0007BE083EB95E00E943A2968EF7AE083EBB2
:101CD00095E00E94F8284091470550914805609191
:101CE000490570914A052AE030E083EB95E00E94B7
:101CF000212A6FED7AE083EB95E00E94F82880912D
:101D00008F0580710E94A70D66EC7AE083EB95E069
:101D10000E94F82880918F0580740E94A70D6DEABB
:101D20007AE083EB95E00E94F82880918F0580721D
:101D30000E94A70D60E97AE083EB95E00E94F82805
:101D400086E495E00E942809AB01BC012AE030E05E
:101D500083EB95E00E94032A6BE87AE083EB95E041
:101D60000E94F82886E495E00E9428099B01AC01B6
:101D700060E472E48FE090E00E94B82CBA01A901FF
:101D80002AE030E083EB95E00E94032A68E87AE0DD
:101D900083EB95E00E943A29CDB7DEB7E5E00C94DD
:101DA000222D8F929F92AF92BF92CF92DF92EF92AD
:101DB000FF92811107C06FE77AE083EB95E00E9404
:101DC0003A292FC090E00E94FD0824E630E040E070
:101DD00050E00E94B82CCA01B9012AE030E040E08E
:101DE00050E00E94B82C49015A016B017C012AE0A5
:101DF00030E0B501A40183EB95E00E94032A6EE276
:101E000083EB95E00E941E292AE030E0B701A6018D
:101E100083EB95E00E94032A63E783EB95E00E9441
:101E20005E29FF90EF90DF90CF90BF90AF909F9092
:101E30008F9008951F93CF93DF9365E77AE083EB4C
:101E400095E00E94F82880916F05813041F46CE59F
:101E50007AE083EB95E00E943A2910E050C082308E
:101E600019F465E47AE0F5CF843019F461E37AE09F
:101E7000F0CF853091F766E27AE0EBCFC12FD0E06A
:101E8000C930D1050CF441C068E3610F83EB95E0E4
:101E90000E941E296EE17AE083EB95E00E94F8280B
:101EA000BE016F5F7F4F4AE050E083EB95E00E94F8
:101EB000E22963E17AE083EB95E00E94F828C159BA
:101EC000DA4FE981E03218F566E07AE083EB95E0DD
:101ED0000E94F8288981803130F06FE373E083EB52
:101EE00095E00E941B2969816F7070E06F5F7F4FE2
:101EF0004AE050E083EB95E00E94EB291F5F809160
:101F00001A05181708F4BACF0FC061E3BECFEF70FF
:101F1000F0E0EE0FFF1FE659FC4F6081718183EB0B
:101F200095E00E944C29EACF6BEE79E083EB95E0D7
:101F30000E94F828809187050E94D10E60ED79E01B
:101F400083EB95E00E94F828809188050E94D10ECD
:101F500065EB79E083EB95E00E94F8288091890594
:101F60000E94D10E6AE979E083EB95E00E94F8289F
:101F700040917F05509180056091810570918205A7
:101F8000411551056105710539F12AE030E083EB17
:101F900095E00E94212A67E679E083EB95E00E94B4
:101FA000F828809183050E942209AB01BC012AE038
:101FB00030E083EB95E00E94212A63E479E083EB33
:101FC00095E00E94F8284AE050E06091840583EB98
:101FD00095E00E94492A06C06AE379E083EB95E028
:101FE0000E943A296DE179E083EB95E00E94F828A0
:101FF00060918505709186054AE050E083EB95E09D
:102000000E94332A60E079E083EB95E00E94F82893
:1020100060917E05603450F470E06F5F7F4F4AE05E
:1020200050E083EB95E00E94EB2906C067EF78E073
:1020300083EB95E00E943A296AED78E083EB95E026
:102040000E94F82880917D0580FF03C063EB71E05A
:1020500002C067EB71E083EB95E00E944C296DEBC9
:1020600078E083EB95E00E94F82880917D058270EE
:102070000E94A70D6EE978E083EB95E00E94F828B6
:1020800080917D0584700E94A70D6FE778E083EB57
:1020900095E00E94F82880917D0588700E94A70D28
:1020A000DF91CF911F9108950F931F93CF93DF93EB
:1020B000209117052F3FA9F56FEF75E083EB95E0B1
:1020C0000E94F82884E793E00E94780D6EED75E099
:1020D00083EB95E00E94F8288091180590911905EE
:1020E0000E94780D6BEA75E083EB95E00E943A2937
:1020F00068E875E083EB95E00E943A2960E775E0B7
:1021000083EB95E00E943A296BE475E083EB95E060
:102110000E943A2983EB95E00E9426290E941A0F1B
:1021200068C012160CF065C0332727FD30958091EA
:102130001A0590E0821793070CF45BC066E375E024
:1021400083EB95E00E94F82860911705772767FDDB
:1021500070954AE050E083EB95E00E94EB296BE03C
:1021600075E083EB95E00E94F82810E008E280918A
:102170001B051817D0F5C12FD0E0CC0FDD1FC45EB2
:10218000DA4F288130E080911705992787FD9095D7
:1021900001972817390739F56BEB71E083EB95E070
:1021A0000E941B294AE050E0602F83EB95E00E94DB
:1021B000122A6FEB71E083EB95E00E941B29E98105
:1021C000EF70F0E0EE0FFF1FE659FC4F6081718168
:1021D00083EB95E00E941B2963EC71E083EB95E0B3
:1021E0000E941B290F5F1F5FC2CF83EB95E00E9407
:1021F0002629DF91CF911F910F910895FF920F93A0
:102200001F93CF93DF93C5E5D5E0F12C8E01888134
:102210008823D1F165EC71E083EB95E00E941B29E6
:102220004AE050E06F2D83EB95E00E94122A62EDA8
:1022300071E083EB95E00E941B292196F801208133
:1022400030E0A0E1B7E20E94722C9B01AC01A091AA
:102250005405B0E00E94812CAB01BC0180914B057C
:1022600090914C05A0914D05B0914E05480F591F16
:102270006A1F7B1F2AE030E083EB95E00E94212A51
:10228000F394F8E1FF12C2CFCDB7DEB7E5E00C94CE
:10229000222D1092B10485E6E2EBF4E0DF011D92FD
:1022A0008A95E9F70895CF93C82F8F3719F08830B2
:1022B00009F045C0E091B104EE23D9F1E150E0937B
:1022C000B104F0E0EE54FB4F10826DE070E083EB60
:1022D00095E00E945906C0E08091B104C81760F4EF
:1022E000EC2FF0E0EE54FB4F608170E083EB95E063
:1022F0000E945906CF5FF0CF60E270E083EB95E07B
:102300000E9459066DE070E083EB95E00E9459064B
:10231000C0E08091B104C81778F5EC2FF0E0EE54DE
:10232000FB4F608170E083EB95E00E945906CF5F20
:10233000F0CF67E083EB95E00E941E291DC08B3132
:1023400019F40E9449111AC08D30C1F08A30B1F0E1
:102350008091B104843668F76C2F70E083EB95E0D0
:102360000E945906E091B10481E08E0F8093B10480
:10237000F0E0EE54FB4FC08380E001C081E0CF91DC
:102380000895CF93C82F0E94602760939A0470939A
:102390009B0480939C0490939D04C093AF04CC2332
:1023A00029F040E051EE60E070E004C040E855E202
:1023B00060E070E083EB95E00E94A82BCF91089538
:1023C00090919E04492F4F7050E0BA016F5F7F4F8C
:1023D000292F30E0E4E035952795EA95E1F762177B
:1023E000730759F0FA01E156FB4F808381E0890FB2
:1023F0008F70907F892B80939E0408956EE770E024
:1024000083EB95E00E94590608951F920F920FB634
:102410000F9211241F932F933F934F935F936F93CA
:102420007F938F939F93AF93BF93CF93DF93EF935C
:10243000FF93C0918600D0918700809159049091BC
:102440005A0420917B04211155C09E01281B390B91
:1024500080918F0590919005A0919105B091920582
:1024600085FD02C036952795253C49E03407B8F133
:1024700040910A0150E060E070E01CE1B695A7953C
:10248000979587951A95D1F70097A105B10521F485
:1024900081E090E0A0E0B0E084179507A607B707B9
:1024A000D8F480910A018F3FB9F040E080910A0191
:1024B000481780F4842F90E0880F991FFC01E55A9B
:1024C000FB4F20813181FC01E55FFE4F318320838A
:1024D0004F5FECCF10927C0410920A010BC02D3B91
:1024E00082E0380720F080910A018031D8F08FEF28
:1024F00080930A01D0935A04C0935904FF91EF913D
:10250000DF91CF91BF91AF919F918F917F916F910B
:102510005F914F913F912F911F910F900FBE0F90A0
:102520001F90189510910A0181E0810F80930A0194
:10253000C9010E94120AE12FF0E0EE0FFF1FE55AD9
:10254000FB4F91838083D6CF83E0809380008AE91C
:102550008093810080918F0586FD05C08091810068
:102560008064809381008FEF9FEF90938900809328
:10257000880080916F00806280936F0008956F30B3
:1025800018F086958058089589E0689F802D112461
:102590000895A0E0B0E0EFECF2E10C94032DC82F19
:1025A0000E94602700910A0410910B0420910C04F2
:1025B00030910D046B017C01C01AD10AE20AF30AC2
:1025C0009701860149E8C41643E1D406E104F10409
:1025D00010F010920E0460930A0470930B04809321
:1025E0000C0490930D0420917B048FEF820F8230B6
:1025F000D8F5E0910E04EE2309F44EC1E13011F458
:1026000082E0B8C1E03108F034C181E08E0F8093E0
:102610000E04F0E0E55AFB4FC083803109F0ACC1F5
:10262000EDE5F4E0213029F4A181A695A6958081FD
:1026300008C080819181A92FA695A695A69596950B
:102640008795A03148F4B0E090E0AA0FBB1FA55FCA
:10265000BE4F11969C938E9310927C04329684E028
:10266000EB36F807F9F688C1233009F005C1E0918F
:102670000E04E11104C0CF3009F07EC10DC1E83174
:1026800048F481E08E0F80930E04F0E0E65AFB4F91
:10269000C08372C1E83109F0ECC0C111EAC040E06A
:1026A00050E0ABE0CA01B3E0880F991FBA95E1F79B
:1026B000A49F9001A59F300D1124F901E55AFB4F0D
:1026C0006081E1817E2F777075956795FC01EE0F33
:1026D000FF1FE55FFE4F71836083F901E45AFB4FF2
:1026E000B081B695B695B695E181FE2FF295FF0FB4
:1026F000F07E6F2F6B2BE695E695E6957E2F777033
:1027000075956795FC01EE0FFF1FE35FFE4F718328
:102710006083F901E35AFB4FB081B295B695B69547
:10272000B370C181DC2FDD0FDD0F6D2F6B2BC295D8
:10273000C695C695C370E281E170EE0FEE0F7E2F55
:102740007C2B75956795FC01EE0FFF1FE15FFE4F37
:1027500071836083F901E15AFB4FB081B695E18145
:10276000FE2FF795FF27F7956F2F6B2BE6957E2FA2
:10277000777075956795FC01EE0FFF1FEF5EFE4FBA
:1027800071836083F901E05AFB4FB081B295BF704D
:10279000E181FE2FF295F07F6F2F6B2BE295EF70AA
:1027A0007E2F777075956795FC01EE0FFF1FED5E2C
:1027B000FE4F71836083F901EF59FB4FB081BB1F5E
:1027C000BB27BB1FC181DC2FDD0F6D2F6B2BCC1FF7
:1027D000CC27CC1FE281E370EE0F7E2F7C2B75950A
:1027E0006795FC01EE0FFF1FEB5EFE4F7183608368
:1027F000F901ED59FB4FB081B695B695E181FE2FF9
:10280000F295FF0FFF0FF07C6F2F6B2BE695E6958F
:102810007E2F777075956795FC01EE0FFF1FE95EBF
:10282000FE4F71836083F901EC59FB4F20812295A3
:10283000269527703181E32FEE0FEE0FEE0F6E2FEE
:10284000622B732F72957695777075956795FC015D
:10285000EE0FFF1FE75EFE4F718360834F5F5F4F98
:102860004230510509F01ECF8091710483FF109210
:102870007C0410920E0480C0243009F07DC0609169
:102880000E0461110BC0C83AB1F4109245051092C4
:10289000440588EA0E94D40681E06CC0613019F4D6
:1028A000C093090404C0623031F4C09308048C2F33
:1028B0000E94D4065AC0E09108042E2F30E0220F67
:1028C000331F462F50E0C9010296841795073CF04C
:1028D000633268F7FA01E85AFB4FC083E8CF2D5FF7
:1028E0003F4F8C2F90E06091440570914505421751
:1028F000530749F4982F88278627972790934505F3
:102900008093440532C06817790769F580910904FE
:10291000813049F5E13118F080E180930804F090AE
:102920000804CCE5D4E000E010E00F15D0F4FE017F
:102930003197808190E0982F88272881822B63E04F
:10294000969587956A95E1F70E94120AF801EE0FB5
:10295000FF1FE55FFE4F918380830F5F1F4F22961D
:10296000E4CF10927C0410920E0480910E04882310
:1029700019F08F5F80930E04CDB7DEB7E8E00C94BA
:102980001F2DE82FF0E0E657FA4FE185E03158F4CB
:10299000F894F0E0EE0FFF1FE55FFE4F20813181DC
:1029A0007894C9010895E03121F0E13131F483E1F7
:1029B00001C082E10E94A228089580E092E008957B
:1029C000A2E2B0E0E6EEF4E10C94F92C9E012F5F58
:1029D0003F4F80E1D9011D928A95E9F766ED71E0DC
:1029E00083EB95E029A33AA30E944C290E94C40CD2
:1029F0001D8A1E8A1F8A188E312C212C00E0812C02
:102A0000912C540170E4472E71EE572E7DE9672E0C
:102A100078E1772EE0E5CE2EE3ECDE2EE12CF12CF2
:102A200084EF91E0A0E0B0E08D8F9E8FAF8FB8A3D0
:102A300080EC91EDA8E9BBE1898F9A8FAB8FBC8FB9
:102A400080E491EEADE9B8E1898B9A8BAB8BBC8BBE
:102A500083EB95E00E94602A892B09F4E1C083EBA7
:102A600095E00E948D2A9C0133272C32310509F410
:102A700042C0ACF42332310509F0ABC019821A828E
:102A80001B821C821D821E821F82188619861A864E
:102A90001B861C861D861E861F86188A60C02434ED
:102AA000310529F02335310509F4B2C092C064E440
:102AB00083EB95E00E941E292AE030E040E451EECD
:102AC0006DE978E183EB95E00E94AC296CE283EB41
:102AD00095E00E941E292AE030E040EC51ED68E9C3
:102AE0007BE183EB95E00E94AC296CE283EB95E0FF
:102AF0000E945E29ADCF0F5F043009F0A9CF298174
:102B00003A814B815C81A8EEB3E00E94812C698BF5
:102B10007A8B8B8B9C8B2D813E814F8158850E94B7
:102B2000812C698F7A8F8B8F9C8F29853A854B8575
:102B30005C852D8F3E8F4F8F58A32D853E854F8509
:102B400058890E94812C6B017C0160323EE473073E
:102B50008105910530F462E38CE10E94D30A00E024
:102B600077CF603345E774078105910510F462E281
:102B7000F3CF60345CE975078105910510F466E2D6
:102B8000EBCF80E5C81683ECD806E104F10410F41D
:102B900062E1E2CF90E6C9169AEED906E104F104AB
:102BA00010F465E1D9CFA0E7CA16A1E1DA06A1E0E9
:102BB000EA06F10410F461E0CFCFB0EACB16B6E834
:102BC000DB06B1E0EB06F10410F463E0C5CF65E08D
:102BD000C3CF10ED180F1A3008F03ACFE1E0F0E063
:102BE000EC0FFD1F24E0029FE00DF11D1124208158
:102BF000318142815381AAE0B0E00E94812C610FB3
:102C0000711D811D911D608371838283938320CF09
:102C100049885A886B887C88812C912C540118CF64
:102C200081149104A104B10489F4C301B2010E948A
:102C3000420B61E070E080E090E00E9483271D8AF3
:102C40001E8A1F8A188E312C22242A948D8D9E8DE7
:102C5000AF8DB8A188169906AA06BB06D0F40E94CB
:102C6000FC0A2D893E894F89588D280F311D411D41
:102C7000511D2D8B3E8B4F8B588F381608F4382EF4
:102C8000821508F4282E3FEF831A930AA30AB30A89
:102C900056C0C301B20128EE33E040E050E00E948C
:102CA000B82CBA01A9012AE030E083EB95E00E943C
:102CB000032A6CE283EB95E00E941E294AE050E073
:102CC000632D83EB95E00E94122A6CE283EB95E082
:102CD0000E941E296D897E898F89988DA501940196
:102CE0000E94B82CBA01A9012AE030E083EB95E0FC
:102CF0000E94032A6CE283EB95E00E941E294AE0C1
:102D000050E0622D83EB95E00E94122A6CE283EB87
:102D100095E00E945E294C0C5D1C6E1C7F1C898D09
:102D20009A8DAB8DBC8D84159505A605B70520F44D
:102D300049885A886B887C88812C912C5401298978
:102D40003A894B895C89283E33404105510509F099
:102D50007FCEA296E2E10C94152DACE1B0E0E3EB5E
:102D6000F6E10C94032D0E9460276B017C0181E049
:102D70000E94B20B14E703E0198361E0CE010196D3
:102D80000E94230D0093A5050E94A10C6AEF70E03C
:102D900080E090E00E9483278091A505833089F42C
:102DA00083EB95E00E94602A892B59F40E946027EA
:102DB0006C197D098E099F096038734C894C9140CC
:102DC000D8F28091A505833009F44FC08FE70E94A7
:102DD000AB0A0E94BE0A8983843511F083E05CC08F
:102DE0000E94BE0A10921805809319050E94BE0A1F
:102DF0002091180530911905280F311D30931905C0
:102E0000209318050E94BE0A80931A050E94BE0AEC
:102E100080931B05813110F7F12C0F2D10E080916C
:102E20001B0590E0880F991F0817190740F40E94AE
:102E3000BE0AF801E45EFA4F8083F394EECF80E798
:102E4000898361E0CE0101960E94230D83E0809387
:102E5000A5050E94A10C62E370E080E090E00E9472
:102E600083278091A505833011F482E015C08FE798
:102E70000E94AB0A0E94BE0A8983803509F0AECF5A
:102E80000FE615E00E94BE0AF80181938F01F5E07C
:102E90000A381F07B9F781E06C96E8E00C941F2D03
:102EA00080911705992787FD9095A92FB92FFC01CF
:102EB0003196EB30F10508F066C0EC5CFF4F0C94E6
:102EC000302D62E778E083EB95E00E943A2984E7B1
:102ED00093E00E94780D6AE578E083EB95E00E942C
:102EE0003A2965E378E083EB95E00E943A296BE0AC
:102EF00078E083EB95E00E943A296AEE77E083EB75
:102F000095E00E943A296DEB77E083EB95E00E9413
:102F10003A2967E977E083EB95E00E943A2963E775
:102F200077E083EB95E00E943A296CE477E083EB4D
:102F300095E00E943A2983EB95E00E9426290E94A1
:102F4000B30D21C06FE277E01AC06AE077E017C0E6
:102F500065EF76E014C066ED76E011C062E976E0D8
:102F60000EC06DE776E00BC068E676E083EB95E097
:102F70000E943A2962E276E002C06CE076E083EBE0
:102F800095E00E943A296AE070E080E090E00E94BB
:102F9000832783EB95E00E94602A892B29F083EB3D
:102FA00095E00E948D2AF5CF0895ACE1B0E0EBEDFD
:102FB000F7E10C94032D909117059F3F09F023C171
:102FC000482F50E0FA013A97EF36F10508F00FC1AB
:102FD000E15CFF4F0C94302D63EE71E0A0C06FEE0A
:102FE00071E083EB95E00E944C2985E789838BE1B2
:102FF000EFE6F5E0DE01129601900D928A95E1F779
:103000006CE1CE0101960E94230D0E94A10C83E089
:103010008093A50568EC70E080E090E00E94832733
:103020008091A505843009F0E2C08FE70E94AB0AC9
:103030000E94BE0A8983853509F0D9C06DEE74E01F
:1030400083EB95E00E943A296FEC74E083EB95E006
:103050000E943A2961EB74E096C067E072E083EB6E
:1030600095E00E944C2989E6898361E0CE010196B2
:103070000E94230D0E94A10C83E08093A50568ECBB
:1030800070E080E090E00E9483278091A505843065
:1030900009F0ADC08FE70E94AB0A0E94BE0A898387
:1030A0008E010E5F1F4F7E014DE1E40EF11C0E9468
:1030B000BE0AF80181938F01EE15FF05C1F78BE180
:1030C000FE013296AFE6B5E001900D928A95E1F7E8
:1030D0008981893409F08BC063E974E083EB95E062
:1030E0000E943A2965E774E083EB95E00E943A2953
:1030F00067E574E048C061E272E083EB95E00E940E
:103100004C298EEF8093170572C0805287508053F0
:1031100090911A05981708F066C060E372E083EB9F
:1031200095E00E944C2963C084E18093170560E21A
:1031300074E029C085E18093170569EE73E023C030
:1031400086E18093170562EB73E01DC087E18093F1
:10315000170568E673E017C088E18093170567E5F7
:1031600073E011C089E18093170563E473E00BC03D
:103170008AE1809317056EE273E005C08BE18093CE
:10318000170566E073E083EB95E00E943A292FC0B3
:103190006CEE72E083EB95E00E943A2980917D0508
:1031A00091E01DC066ED72E083EB95E00E943A2944
:1031B00080917D0592E013C061EC72E083EB95E0B5
:1031C0000E943A2980917D0594E009C066EA72E088
:1031D00083EB95E00E943A2980917D0598E089274C
:1031E00080937D058FEF809317050E94541083EB29
:1031F00095E00E94602A892B09F45BC183EB95E07E
:103200000E948D2AF4CF0E945311882309F451C1E2
:103210008091B104811104C08FEF8093170541C1E3
:1032200040E050E060E070E082EB94E00E94A72D67
:1032300040911705042F112707FD1095212F312FDD
:10324000F8013197EB31F10508F01BC1E255FF4F52
:103250000C94302D552747FD509520911A0530E0EC
:10326000241735070CF40DC18B019C010150110985
:1032700021093109003211052105310558F0C090AE
:103280001B05EDE1F5E0F12CD12CA8E2EA2E41502E
:1032900051090FC0FA01E159FA4F61506083D9C05A
:1032A000DF0111972C9130E02417350729F0F394B2
:1032B0003296FC10F5CFCBC00E2D10E020E030E0B0
:1032C000061717072807390741F42081DA01A159A9
:1032D000BA4F11962C93DD24D394E394E8CF6F3F3B
:1032E00071058105910511F008F0CBC06093870549
:1032F000B0C06F3F71058105910511F008F0C1C0A4
:1033000060938805A6C06F3F71058105910511F096
:1033100008F0B7C0609389059CC02091B204206278
:103320002037E9F440E050E060E070E083EB94E0A7
:103330000E94A72D9B01AC01DC01CB010197A109E3
:10334000B1090897A105B10508F0AEC0A4EDB0E33E
:103350000E94812C6A5E7C4A8A46954E24C026369D
:10336000E9F440E050E060E070E083EB94E00E941C
:10337000A72D9B01AC01DC01CB010197A109B1098B
:103380000797A105B10508F08FC0A8EAB1E60E9431
:10339000812C645E7C438E46944E05C06115710598
:1033A0008105910579F08B019C010054114E2D4946
:1033B00038410138F0EF1F07FAEF2F07F2E03F071F
:1033C00008F05FC060937F0570938005809381054E
:1033D000909382053EC06F3F71058105910511F004
:1033E00008F04FC06093830534C08B019C010150ED
:1033F0001109210931090F3F11052105310508F097
:1034000040C06093840525C08B019C01045C194079
:10341000210931090D344DE114072105310528F446
:10342000709386056093850514C06115710581054B
:10343000910521F48FEF80937E050BC061347105F7
:1034400081059105F0F4615060937E0502C0DD2096
:10345000C1F08091B00481111AC080914F05909104
:103460005005A0915105B09152050196A11DB11DC5
:1034700080934F0590935005A0935105B09352054A
:1034800006C062E472E083EB95E00E944C290E9442
:1034900049118FEF809317056AE083EB95E00E9456
:1034A0005E290E94541005C061E070E080E090E069
:1034B0007ACF6C96E8E00C941F2D6AE572E083EBFE
:1034C00095E00E943A2962E472E083EB95E00E9465
:1034D0003A2983EB95E00E94602A892B31F083EB37
:1034E00095E00E948D2A0E94D5170E94AD16823069
:1034F00029F0833051F46DE072E002C064E272E0C2
:1035000083EB95E00E943A2908958FEF8093170589
:103510001092B0040E945410809117058E3F69F0FC
:1035200083EB95E00E94602A892BB1F383EB95E051
:103530000E948D2A0E94D517EFCF08950F931F93F5
:10354000109117051F3F09F0D1C0893409F457C005
:1035500000F5883309F468C058F4803309F476C064
:1035600008F060C08B3109F440C08132B1F1B8C0BD
:10357000813409F486C030F4893309F465C080349D
:1035800061F1AEC0823409F48DC0863409F447C0BD
:10359000A7C0823609F486C078F4883531F128F462
:1035A0008235C1F18335E1F09BC08A3509F493C0BF
:1035B000813609F466C094C0823761F128F48636FA
:1035C00071F18936E1F08CC0883779F08A3709F4D7
:1035D00082C0833709F084C003C063EE71E015C078
:1035E0000E94DF0860E672E004C00E94E8086AE713
:1035F00072E083EB95E00E944C298EEF6FC00E9431
:10360000B7070E94260869E972E083EB95E00E9403
:103610004C2966C00E94460862EB72E0F6CF0E9419
:10362000FE105EC080535AC06AEF71E083EB95E0F4
:103630000E943A2990916E0588E0890F8871977EE3
:10364000892B80936E051AC089E048C067EE71E04F
:1036500083EB95E00E943A2980918F059091900527
:10366000A0919105B091920520E1822780938F056A
:1036700090939005A0939105B09392051093170530
:103680002FC061ED71E083EB95E00E943A298091B3
:103690008F0590919005A0919105B091920540E41D
:1036A000842710C060EC71E083EB95E00E943A291A
:1036B00080918F0590919005A0919105B091920510
:1036C00020E2822780938F0590939005A093910527
:1036D000B093920502C00E945D1A8FEF8093170588
:1036E000809117058E3F09F0D4C0DDC00E945311B0
:1036F000882309F4D8C08091B104811104C08FEFF0
:1037000080931705C6C040E050E060E070E082EBB7
:1037100094E00E94A72D00911705112707FD109531
:10372000212F312FF8013197E930F10508F0B4C0AD
:10373000E753FF4F0C94302D8B019C010154114E27
:103740002D4938410F37104F2A4F324008F0A4C09E
:1037500060934B0570934C0580934D0590934E05F7
:1037600077C060934F0570935005809351059093F7
:10377000520581E08093B0046BC06830710581050B
:10378000910508F089C06093530562C08B019C01CC
:1037900001501109210931090A30110521053105AE
:1037A00008F07AC06093540553C061EB71E082EB7E
:1037B00094E00E94E12E10E0009799F00E94BB2E49
:1037C000009779F0183130F4E12FF0E0EA5BFA4F1E
:1037D00087871F5F61EB71E080E090E00E94E12E3F
:1037E000EBCF1831A8F5E12FF0E0EA5BFA4F17862E
:1037F0001F5FF7CF653071058105910508F04CC05A
:1038000060936D0525C08B019C01015011092109B0
:1038100031090630110521053105F0F520916E05BD
:10382000287F262B20936E0513C08B019C0101502D
:103830001109210931090115124C2140310560F5AA
:1038400060934705709348058093490590934A0516
:103850008091B004811113C080914F059091500563
:10386000A0915105B09152050196A11DB11D809303
:103870004F0590935005A0935105B09352050E94B7
:1038800049118FEF809317056AE083EB95E00E9462
:103890005E290E94501707C062E472E083EB95E056
:1038A0000E944C29ECCF1F910F9108958FEF8093C8
:1038B00017051092B0040E945017809117058E3F93
:1038C00069F083EB95E00E94602A892BB1F383EBCA
:1038D00095E00E948D2A0E949E1AEFCF6AE070E068
:1038E00080E090E00E94832783EB95E00E94602AAD
:1038F000892B29F083EB95E00E948D2AF5CF08955E
:10390000CF93C82F682F83EB95E00E94BA2A90913D
:103910003C059C2790933C05CF910895A1E0B0E031
:10392000E4E9FCE10C94092D99830E94801C9981A3
:10393000892F0E94801C2196E2E00C94252D1F9374
:10394000CF93DF93182FEB0110923C0565EB70E0ED
:1039500083EB95E00E94590662E670E083EB95E008
:103960000E945906812F0E94801CCE010E948E1C4D
:10397000DF91CF911F91089560913C0583EB95E015
:103980000E94BA2A0895A1E2B0E0E9ECFCE10C94AF
:10399000052D7B018A018B3009F42DC108F03FC051
:1039A000853009F49BC010F5823009F47EC058F4CC
:1039B000813009F02FC269E270E081E00E949F1C13
:1039C00006E415E068C0833009F480C0843009F053
:1039D00021C261E070E084E00E949F1C81E00E94AF
:1039E000801C0E94BC1C0E94E0141EC2883009F496
:1039F0009BC070F4863009F48DC0873009F00AC28C
:103A000061E070E087E00E949F1C80911A0508C267
:103A1000893009F491C08A3009F4C3C0FBC18936EA
:103A200009F468C178F4863609F419C120F48536A2
:103A300009F401C1EFC1873609F425C1883609F4BC
:103A40002AC1E8C18C3609F49EC190F48A3609F483
:103A50005BC18B3609F0DEC161E070E08BE60E944D
:103A60009F1CF80180810E940E080E94E808BDC1D9
:103A70008D3609F4BCC1873C09F0CCC161E070E02F
:103A800087EC0E949F1C81E00E94801C0E94BC1C4D
:103A900010923D05C9C1F80181918F010E94801CDF
:103AA000F5E00F361F07B9F7BDC16BE170E082E0AA
:103AB0000E949F1C0FE615E0F80181918F010E9482
:103AC000801CF5E00A381F07B9F7ACC161E070E06F
:103AD00083E00E949F1C0E94AD16A2C160911B054D
:103AE00070E0660F771F85E00E949F1C0CE115E0D7
:103AF00080911B0590E0880F991F98012C5135404B
:103B00002817390708F08EC1F80181918F010E94B2
:103B1000801CEECF62E070E086E00E949F1C84E78C
:103B200093E00E948E1C7EC161E070E088E00E94FC
:103B30009F1C8091A30574C186E6898361E0CE0154
:103B400001960E94230D0E94A10C83E08093A5059D
:103B500068EC70E080E090E00E9483278091A505EA
:103B60008430D9F48FE70E94AB0A0E94BE0A898391
:103B7000863469F460E270E089E00E949F1C10E2E4
:103B80000E94BE0A0E94801C1150D1F74BC161E017
:103B900070E089E00E949F1C28C161E070E089E02C
:103BA0003CC169E170E08AE00E949F1C10928A0586
:103BB0002091A40580918F0590919005A091910589
:103BC000B0919205222311F0806801C08F77809315
:103BD0008F0590939005A0939105B09392050AE804
:103BE00015E0F80181918F010E94801CF5E0033AF5
:103BF0001F07B9F717C161E270E08BE00E949F1CBC
:103C000080917C048F3F39F080917C0491E0980F83
:103C100090937C0402C080917C040E94801C10E080
:103C2000812F0E94C1140E943D0A0E948E1C1F5FBA
:103C30001031B1F7F7C061E070E085E60E949F1C8B
:103C400089E2E816F10409F0EAC0D801E6E4F5E0FB
:103C50008D91819385E0EF36F807D1F7C6C061E01A
:103C600070E086E60E949F1CEBE1EE16F10409F07D
:103C7000D6C0D801EFE6F5E08D91819385E0EA3872
:103C8000F807D1F7B2C061E070E087E60E949F1CA0
:103C90000E94DF08AAC061E070E088E60E949F1CD5
:103CA00085E789838BE1EFE6F5E0DE01129601906E
:103CB0000D928A95E1F76CE1CE0101960E94230DE9
:103CC0000E94A10C83E08093A50560E273E080E090
:103CD00090E00E9483278091A505843009F09FC061
:103CE0008FE70E94AB0A0E94BE0A8983853509F0DE
:103CF00096C07BC061E070E089E60E949F1C0E9434
:103D0000B7070E94260871C061E070E08AE60E9451
:103D10009F1C89E6898361E0CE0101960E94230DF4
:103D20000E94A10C83E08093A50560E273E080E02F
:103D300090E00E9483278091A505843009F06FC030
:103D40008FE70E94AB0A0E94BE0A89838E010E5F34
:103D50001F4F7E01EDE1EE0EF11C0E94BE0AF8013C
:103D600081938F01EE15FF05C1F78BE1FE013296BD
:103D7000AFE6B5E001900D928A95E1F7898189342B
:103D800009F04DC032C061E070E08CE60E949F1CDB
:103D9000F0E2EF16F10461F487E6898380E2F8012E
:103DA000DE01129601900D928A95E1F761E203C05F
:103DB00087E4898361E0CE0101960E94230D0E9471
:103DC000A10C83E08093A5056CE474E080E090E0B2
:103DD0000E9483278091A505843009F58FE70E9412
:103DE000AB0A0E94BE0A8734D1F481E019C061E0B9
:103DF00070E08DE60E949F1C89E1E816F10479F4D9
:103E0000D801EAE8F5E08D91819385E0E33AF8077F
:103E1000D1F7EBCF61E070E08AEC0E949F1C80E05C
:103E20000E94801C0E94BC1CA196E6E00C94212DEF
:103E3000A0E0B0E0EEE1FFE10C94032DCCE9D3E08B
:103E400014E606E035E0F32E44E0E42E53E0D52EF0
:103E500062E0C62E83EB95E00E94602A892B09F46C
:103E60009BC083EB95E00E948D2A282F8093070446
:103E70004091060450E04730510560F7FA01EE52D8
:103E8000FF4F0C94302D853B29F781E08093060489
:103E9000E1CF823609F07DC0C0920604DBCF80936B
:103EA000050480930404D0920604D4CF9C013327E8
:103EB0003093030420930204909104049827909374
:103EC0000404E0920604C6CF382F22274091020452
:103ED00050910304242B352B3093030420930204C8
:103EE00090910404982790930404F09206042536D8
:103EF000310508F4AFCF61E070E08CEC0E949F1CAC
:103F000081E00E94801C0E94BC1C43C020910004E0
:103F100030910104F901E456FC4F80839091040430
:103F2000982790930404C90101969093010480930B
:103F3000000420910204309103048217930708F4CF
:103F400089CF0093060486CF8091040482130BC0AE
:103F500060910004709101044CE953E080910504E4
:103F60000E94C31C0DC062E070E08BEC0E949F1C9D
:103F7000809105040E94801C80913C050E94801C59
:103F8000FE01812F11928A95E9F710920104109297
:103F90000004109206045ECFCDB7DEB7E8E00C94C3
:103FA0001F2D81E080933D0580913D05882349F0D8
:103FB00083EB95E00E94602A892BB1F30E94181FC1
:103FC000F3CF0895AAE2B0E0E8EEFFE10C94012DF2
:103FD0000E9454276B017C0181E00E94B20B83EBAD
:103FE00095E00E94602A892B29F083EB95E00E94DE
:103FF0008D2AF5CF5E9811E072E6B72EE9E2AE2E7B
:1040000003E00E9454276C197D098E099F09693CC1
:10401000710581059105D0F11123C1F10E9454274A
:104020006B017C015D9A80ED97E00E947006B98279
:10403000E6E4F5E0DE0112968A2D01900D928A9554
:10404000E1F76AE2CE0101960E94230D5D9880E0BF
:1040500090E00E9470060093A5050E94A10C62E307
:1040600070E080E090E00E9483278091A505843075
:1040700061F40093A5058FE70E94AB0A0E94BE0A77
:1040800011E0823419F410E001C011E08EE00E94CA
:104090007928892B81F411E00EC05E9A5D9A83EB3A
:1040A00095E00E948D2A8D309105A9F05CF40A9765
:1040B00091F05E985D9883EB95E00E94602A892BD1
:1040C00061F79FCF8332910579F08234910589F7AA
:1040D0000E94D11FEECF62EB71E083EB95E00E946E
:1040E0003A290E94561CE5CF0E94E014E2CF8F923D
:1040F0009F92AF92BF92CF92DF92EF92FF921F9367
:10410000CF93DF938EE00E947928892B09F078C045
:1041100068EC70E080E090E00E94832780E090E00F
:104120000E9470060E9454274B015C016B017C01C8
:1041300080ECC80E82E1D81EE11CF11C0E945427BD
:104140006C157D058E059F0530F48EE00E94792860
:10415000892BA1F353C08EE00E947928892B09F0A6
:104160004DC080ED97E00E9470060E9454276B01BD
:104170007C01D0E0C1E088E4880E86E2981EA11C94
:10418000B11C11E08EE00E947928892B21F58C1456
:104190009D04AE04BF0430F480ED97E00E947006E9
:1041A000D1E0F0CF0E9454276C197D098E099F0938
:1041B000693C71058105910528F30E9454276B0124
:1041C0007C01C12719F080ED97E002C080E090E00B
:1041D0000E947006D7CF80E090E00E947006DD2339
:1041E00049F08091A3058F5F83700E940E080E94A2
:1041F000E80806C00E9446080E94DF080E94E21FED
:10420000DF91CF911F91FF90EF90DF90CF90BF9003
:10421000AF909F908F900895CF92DF92EF92FF9290
:1042200080E00E94BA060E94910661E089E00E9447
:104230000D2860E089E00E94462861E086E00E9447
:104240000D2861E085E00E940D2860E08EE00E946C
:104250000D2860E088E00E940D2861E088E00E945F
:10426000462861E081E10E940D2860E081E10E9422
:1042700046280E94610640E052EC61E070E083EB6A
:1042800095E00E94A82B0E9401080E94E8080E9465
:10429000A4128FEF80937C040E94A60678940E945B
:1042A00054276B017C0180917C048F3F59F40E945C
:1042B00054276C197D098E099F09603D774081055F
:1042C000910588F380ED97E00E94700661E08EE032
:1042D0000E9446285E9A83EB95E00E94602A892B13
:1042E00029F083EB95E00E948D2AF5CF6FEC72E008
:1042F00083EB95E00E941B2984E793E00E94780DF0
:1043000066EE72E083EB95E00E941B294AE050E0E4
:1043100064E070E083EB95E00E94EB2962E370E0DB
:1043200080E090E00E94832783EB95E00E94602A62
:1043300004970CF183EB95E00E948D2A823491055D
:10434000D1F483EB95E00E948D2A8E34910599F487
:1043500083EB95E00E948D2A8434910561F483EB10
:1043600095E00E948D2A819731F480E090E00E94D0
:1043700070060E94E21F40914705509148056091E8
:10438000490570914A05DB01CA010197A109B109EC
:104390000497A105B10568F440937B04433029F4E8
:1043A00040EA56E861E070E004C040E052EC61E0B1
:1043B00070E083EB95E00E94A82B0E9477205E9826
:1043C00080E090E00E9470060E94A4121092970470
:1043D00080918F0583FF11C080915B05882351F088
:1043E00080916205882331F080916905882311F05E
:1043F00087E001C085E08093970480E00E94B20BC3
:10440000809198040E94E60A0E94A10C1092110467
:104410001092100410920F04F12C8091A3058F15B7
:10442000B0F062E370E080E090E00E94832780EDCE
:1044300097E00E94700662E370E080E090E00E94E6
:10444000832780E090E00E947006F394E6CF80918D
:104450006E0584FF08C0982F987181E0983109F0AB
:1044600080E00E94C1118FE00E94BA06FF90EF9099
:10447000DF90CF900895EF92FF920F931F93CF9309
:10448000DF938C016EE770E083EB95E00E945906A4
:10449000E801F12CF0E2EF2E8E0188818D578230F9
:1044A00048F46DE770E083EB95E00E94590688813F
:1044B0008E2588832196F801608183EB95E00E9428
:1044C000BA2AF394F9E0FF12E7CF6EE770E083EBCE
:1044D00095E00E945906CDB7DEB7E6E00C94212D99
:1044E000A9E0B0E0E6E7F2E20C94092D909199047E
:1044F00091110EC09EEF99838A836B8350E055958E
:1045000047954C832D83198618861F821E822EC0E4
:1045100040919E04842F90E0B4E095958795BA95DC
:10452000E1F7242F2F7030E08217930719F18DEFF8
:1045300089831B82FE01349650E0842F90E0A4E032
:1045400095958795AA95E1F7242F2F7030E0821773
:10455000930749F0DC01A156BB4F8C918193405FDA
:104560005F5F563051F740939E045A83CE01019607
:104570000E943B228091990490E0019666E070E0F1
:104580000E94A42C809399042996E2E00C94252D96
:10459000A0E0B0E0EEECF2E20C94022D6C016EE7CC
:1045A00070E083EB95E00E9459068601E12CF12C26
:1045B000C0E0D0E030E2B32EF801608183E8860FDE
:1045C000823078F46DE770E083EB95E00E94590645
:1045D000F80160816B2570E083EB95E00E9459063D
:1045E00004C083EB95E00E94BA2AE114F10459F06B
:1045F000F80180819E01280F311DC901C92FDD27D7
:10460000C80FD91FDD273FEFE31AF30A89E0E81648
:10461000F10459F028E0E216F10421F48C2F809582
:10462000F60180870F5F1F4FC7CFCDB7DEB7E9E038
:104630000C941E2DA9E0B0E0E0E2F3E20C94092D09
:10464000E82F362F8091990490E0019664E270E0A3
:104650000E94A42C8093990458E9598350E15A830D
:10466000813089F048F08230B9F08330D9F48B83FF
:1046700081EF8C833D8319C085E08B8381EF8C8330
:104680002F5F2D8312C08B8381EF8C8384E6489F3C
:10469000A00111245D8309C084E08B8381EF8C83AA
:1046A000ED8303C00E94FE1104C0CE0101960E945A
:1046B000C8222996E2E00C94252DA2E0B0E0E3E6C2
:1046C000F3E20C94FE2C182F762E2A8349830E9445
:1046D00060276B017C018091AF0480909A049090D8
:1046E0009B04A0909C04B0909D042A81498188235A
:1046F000C1F0D701C60188199909AA09BB094C0163
:104700005D0191EE89169EE29906A104B10420F1A3
:10471000241708F4422F202F672D812F0E941A237F
:1047200013C0D701C60188199909AA09BB094C0110
:104730005D0191E3891695E79906A104B10460F043
:10474000672D812F0E947022C0929A04D0929B0400
:10475000E0929C04F0929D042296EDE00C941A2DB8
:10476000A2E2B0E0E6EBF3E20C94FF2C8CE00E94B6
:10477000CD0A81110DC06EEE72E083EB95E00E94D0
:104780004C295E9A80E00E94B20B0E94A10C5E98B8
:1047900083EB95E00E94602A892B01F183EB95E081
:1047A0000E948D2A90917B04992319F00E94C912CE
:1047B000EFCF4091100450E09A012F5F3F4F2F71CF
:1047C00033276091110470E02617370709F3FA01C7
:1047D000E55EFB4F808320931004DACF8091A5051E
:1047E000843009F086C00E9460276115710581053B
:1047F000910549F06093890470938A0480938B0437
:1048000090938C040CC081E090E0A0E0B0E0809335
:10481000890490938A04A0938B04B0938C048091B4
:104820007F049091800481609093800480937F0442
:1048300083E08093A5058FE70E94AB0A0BE314E0A9
:104840000E94BE0AF80181938F01F4E004341F072F
:10485000B9F72091440480913B04982F922796FF4A
:104860003BC090E4922790934404982F9873983318
:10487000F1F410E0212F30E080913B04877090E04C
:10488000821793074CF11F5F20916E05812F90E0F6
:10489000FC01E55CFB4F24FF04C080810E94E01115
:1048A000E9CF608183EB95E00E94BA2AE3CF8F7352
:1048B00099F480913C048093880480913D04809316
:1048C000860480913E04809385048091410490E0A9
:1048D00090937E0480937D0480910F04813019F4BD
:1048E00082E080930F0480910F04833011F41092C2
:1048F0000F040E9460276B017C01809181049091DC
:104900008204A0918304B09184040097A105B105AD
:10491000C9F0A7019601281B390B4A0B5B0BDA0182
:10492000C901883B9B40A105B10560F00E94FC0ACB
:104930008093870410928104109282041092830461
:104940001092840480918D0490918E04A0918F0424
:10495000B091900446015701881A990AAA0ABB0A25
:1049600086E495E00E94280986169706A806B906EF
:1049700008F4A4C0C0928D04D0928E04E0928F04FB
:10498000F09290040E94570680917C048830A0F039
:1049900080918F0590919005A0919105B09192051D
:1049A0006CE1B695A795979587956A95D1F7892B70
:1049B0008A2B8B2B09F0A7C180917C048F5F809399
:1049C0007C048091890490918A04A0918B04B09119
:1049D0008C040097A105B105F1F0C81AD90AEA0ABA
:1049E000FB0A86E495E00E9428096C157D058E057A
:1049F0009F0508F002C180918F0584FD04C080ED01
:104A000097E00E9470061092890410928A04109216
:104A10008B0410928C0490914404907C90934404F5
:104A2000509110048091110420910F04581709F43B
:104A300001C1223009F0FEC0905890934404E091E7
:104A40006E05E770F0E0E45BFC4F6081693008F0D0
:104A5000D9C0615040E04613D7C08093110487E36A
:104A6000840F90914404892B809344044093120452
:104A700083E080930F045D9A9091970491112DC16A
:104A8000809198040E94E60AE0916E05E770F0E0DC
:104A9000E45BFC4F608184E494E00E94DC0CE091D4
:104AA0009804EF5FE0939804E83109F429C1F0E03D
:104AB000EA5BFA4F8785882309F422C10E944B0DD7
:104AC000813069F580916E05887149F180917F048C
:104AD00090918004880F991F9093800480937F04A5
:104AE00083E08093A5050E94A10C0E94602760933B
:104AF0008104709382048093830490938404672BD1
:104B0000682B692B61F481E090E0A0E0B0E0809335
:104B1000810490938204A0938304B09384048091D1
:104B20006E0584FF1FC080917F04909180048E7F6A
:104B30000E945E0A182F60917D04809188040E9473
:104B4000BF12482F612F8091870449A30E94BF1292
:104B50000091A305282F49A16091850480918604C6
:104B60000E945D235D98809195048130C1F018F01A
:104B70008230B1F1D1C08EE00E947928892B09F0F2
:104B8000CBC081E0809395040E94542760939104E8
:104B9000709392048093930490939404BDC08EE02C
:104BA0000E947928892B31F50E945427C0909104E6
:104BB000D0909204E0909304F09094046C197D09D5
:104BC0008E099F09693E73408105910508F4A4C0D0
:104BD00082E08093950480ED97E00E9470069CC06F
:104BE0008EE00E947928892B09F496C080E090E03D
:104BF0000E947006109295048FC080E090E00E94A1
:104C0000700609CF68E026CF851709F426CF4F5FDD
:104C1000242F30E090E0F901EC5BFB4FDC01A55E56
:104C2000BB4F7C917083F901EE5EFB4F7083019660
:104C30008F7111CF2430B1F42091120483E194E0FC
:104C4000A5E4B4E0FC013E2F381B321718F4319173
:104C50003D93F9CF87E3820F90914404892B809391
:104C6000440406CF80919504823069F4916090935A
:104C700044045E9A53E9E52E55E0F52E8E010F5F50
:104C80001F4FB80110C05E9880910F04811103C0BE
:104C900081E080930F0480910F04833059F784E002
:104CA00080930F04E7CFF70181917F0169A37AA375
:104CB0000E94C114F801819391938F0169A17AA197
:104CC000F3EAEF16F5E0FF0671F780916E0545E413
:104CD00054E087700E94AD09CECE809153058823A1
:104CE00009F4CECE2091960431E0320F3093960431
:104CF000291303C01092960481500E94AD0BC0CEC0
:104D000010929804DBCE80917C04883009F45E9A7E
:104D100089E080937C04D2CEA296ECE00C941B2D0B
:104D20008230E8F4E82FF0E0EE0FFF1FEA55FA4F6B
:104D300071836083813041F0809169008C7F842B86
:104D400080936900E89A089580916900440F551F87
:104D5000440F551F837F842B80936900E99A08953F
:104D60001F920F920FB60F9211242F933F934F93E0
:104D70005F936F937F938F939F93AF93BF93EF93C3
:104D8000FF938091A6059091A705892B29F0E091CA
:104D9000A605F091A7050995FF91EF91BF91AF91FD
:104DA0009F918F917F916F915F914F913F912F9143
:104DB0000F900FBE0F901F9018951F920F920FB675
:104DC0000F9211242F933F934F935F936F937F9391
:104DD0008F939F93AF93BF93EF93FF938091A80519
:104DE0009091A905892B29F0E091A805F091A905DA
:104DF0000995FF91EF91BF91AF919F918F917F9115
:104E00006F915F914F913F912F910F900FBE0F9037
:104E10001F9018951F920F920FB60F9211242F9387
:104E20003F938F939F93AF93BF938091AB059091E6
:104E3000AC05A091AD05B091AE053091AA0523E077
:104E4000230F2D3720F40196A11DB11D05C026E8C2
:104E5000230F0296A11DB11D2093AA058093AB05D7
:104E60009093AC05A093AD05B093AE058091AF05CE
:104E70009091B005A091B105B091B2050196A11D28
:104E8000B11D8093AF059093B005A093B105B09389
:104E9000B205BF91AF919F918F913F912F910F904C
:104EA0000FBE0F901F9018952FB7F8946091AB0527
:104EB0007091AC058091AD059091AE052FBF08951E
:104EC0003FB7F8948091AF059091B005A091B105DE
:104ED000B091B20526B5A89B05C02F3F19F00196E9
:104EE000A11DB11D3FBF6627782F892F9A2F620F12
:104EF000711D811D911D42E0660F771F881F991F4C
:104F00004A95D1F70895CF92DF92EF92FF92CF9317
:104F1000DF936B017C010E946027EB01C114D10477
:104F2000E104F10479F00E9460276C1B7D0B683E60
:104F30007340A0F381E0C81AD108E108F108C85114
:104F4000DC4FECCFDF91CF91FF90EF90DF90CF90CF
:104F50000895789484B5826084BD84B5816084BDF1
:104F600085B5826085BD85B5816085BDEEE6F0E0E2
:104F7000808181608083E1E8F0E01082808182603E
:104F80008083808181608083E0E8F0E080818160BF
:104F90008083E1EBF0E0808184608083E0EBF0E0EF
:104FA000808181608083EAE7F0E080818460808393
:104FB000808182608083808181608083808180683D
:104FC00080831092C1000895833081F028F48130ED
:104FD00099F08230A1F008958630A9F08730B9F0B9
:104FE0008430D1F4809180008F7D03C08091800057
:104FF0008F7780938000089584B58F7702C084B541
:105000008F7D84BD08958091B0008F7703C080911B
:10501000B0008F7D8093B0000895CF93DF9390E030
:10502000FC01ED50F44F2491FC01E95FF34F8491B2
:10503000882349F190E0880F991FFC01E15DF34F4F
:10504000A591B4918B5D934FFC01C591D4919FB70D
:10505000611108C0F8948C91209582238C938881EB
:1050600082230AC0623051F4F8948C91322F30952B
:1050700083238C938881822B888304C0F8948C913D
:10508000822B8C939FBFDF91CF910895A1E0B0E078
:10509000ECE4F8E20C94072D282F30E0F901E152FE
:1050A000F44F8491F901ED50F44F1491F901E95F47
:1050B000F34F04910023C9F0882321F069830E94F3
:1050C000E4276981E02FF0E0EE0FFF1FEB5DF34F67
:1050D000A591B4919FB7F8948C91611103C010957C
:1050E000812301C0812B8C939FBF2196E4E00C9417
:1050F000232DCF93DF93282F30E0F901E152F44FB5
:105100008491F901ED50F44FD491F901E95FF34F27
:10511000C491CC2391F081110E94E427EC2FF0E0A0
:10512000EE0FFF1FE55EF34FA591B4912C912D2357
:1051300081E090E021F480E002C080E090E0DF9127
:10514000CF9108958E3008F08E50877020919D0188
:1051500090E4299F90011124822B80937C00809100
:105160007A00806480937A0080917A0086FDFCCF7B
:10517000809178002091790090E0922B0895A0E032
:10518000B0E0E5ECF8E20C94032D6C017A01EB0140
:10519000E60EF71E00E010E0CE15DF0561F0699124
:1051A000D601ED91FC910190F081E02DC6010995A9
:1051B000080F191FF1CFC801CDB7DEB7E8E00C9496
:1051C0001F2D6115710589F0DB010D900020E9F7B5
:1051D000AD0141505109461B570BDC01ED91FC918B
:1051E0000280F381E02D0995089580E090E0089514
:1051F000EF92FF920F931F93CF93DF938C01FB01EC
:10520000C0E0D0E064917F018FEFE81AF80A6623CE
:1052100061F0D801ED91FC910190F081E02DC80181
:105220000995C80FD91FF701EDCFCE01CDB7DEB775
:10523000E6E00C94212D0E94E1280895DC01ED9117
:10524000FC910190F081E02D099508950F931F9333
:10525000CF93DF93EC016DE00E941E298C016AE080
:10526000CE010E941E29800F911FDF91CF911F91C7
:105270000F9108950F931F93CF93DF93EC010E943A
:10528000F8288C01CE010E942629800F911FDF9102
:10529000CF911F910F9108950F931F93CF93DF9399
:1052A000EC010E94E1288C01CE010E942629800F8A
:1052B000911FDF91CF911F910F9108950F931F932D
:1052C000CF93DF93EC010E941E298C01CE010E9436
:1052D0002629800F911FDF91CF911F910F91089583
:1052E000A1E2B0E0E6E7F9E20C94FF2C7C01C42EC9
:1052F000E52FCB01D22E19A221E02D1510F02AE0C6
:10530000D22E8E010F5D1F4F8D2C912CA12CB12C14
:105310006C2D7E2FA50194010E94B82C8C2DD29E5D
:1053200080191124015011098A3010F4805D01C0E8
:10533000895CF8018083211531054105510521F073
:10534000C22EE32FCA01E4CFB801C7010E94E128B1
:10535000A196ECE00C941B2DA0E0B0E0E2EBF9E2AA
:105360000C94032DEC016A017B012115310541F4F8
:10537000E881F9810190F081E02D642F09951DC02D
:105380002A303105A9F477FF12C06DE20E941E2970
:105390008C0144275527BA014C195D096E097F0914
:1053A0002AE0CE010E947029800F911F06C02AE0DA
:1053B000B701A601CE010E947029CDB7DEB7E8E0A3
:1053C0000C941F2D9A01AB01662757FD6095762F2F
:1053D0000E94AC2908950F931F93CF93DF93EC01A4
:1053E0009A01AB01662757FD6095762F0E94AC2984
:1053F0008C01CE010E942629800F911FDF91CF9151
:105400001F910F9108952115310549F4DC01ED91AB
:10541000FC910190F081E02D642F099508950E9480
:10542000702908959A01462F50E060E070E00E94D4
:10543000032A08959A01AB0160E070E00E94032AFC
:1054400008950F931F93CF93DF93EC010E94032ADB
:105450008C01CE010E942629800F911FDF91CF91F0
:105460001F910F9108950F931F93CF93DF93EC013A
:105470009A01AB0160E070E00E94032A8C01CE012A
:105480000E942629800F911FDF91CF911F910F91CC
:1054900008950F931F93CF93DF93EC019A01462F4A
:1054A00050E060E070E00E94032A8C01CE010E946F
:1054B0002629800F911FDF91CF911F910F910895A1
:1054C000FC0124853585F901E05CFF4F80819181E5
:1054D000F901EE5BFF4F20813181821B930B8F73AB
:1054E00099270895FC0184859585FC01E05CFF4FB8
:1054F00040815181FC01EE5BFF4F208131814217D9
:10550000530741F00190F081E02DE80FF91F8081F1
:1055100090E008958FEF9FEF0895FC0184859585B5
:10552000FC01E05CFF4F40815181FC01EE5BFF4FCD
:10553000208131814217530779F0A081B181A80FF2
:10554000B91F8C91208131812F5F3F4F2F733327FB
:105550003183208390E008958FEF9FEF0895FC0141
:1055600081A1882329F0A489B5898C9186FFFBCF7E
:1055700011A20895CF93DF93FC0126853785D901C9
:10558000A05CBF4F8D919C91119701968F739927C5
:10559000E901CE5BDF4F4881598184179507D9F324
:1055A0000D90BC91A02DA20FB31F6C93A685B7855B
:1055B000A05CBF4F11969C938E93A689B7892C91BE
:1055C00081E090E0078C02C0880F991F0A94E2F7EF
:1055D000282B2C9381E081A30488F589E02D80811C
:1055E0008064808381E090E0DF91CF9108950895F9
:1055F0001F920F920FB60F9211242F933F934F9348
:105600008F939F93EF93FF938091C00082FD1CC006
:105610004091C6008091590690915A0601968F7369
:10562000992720915B0630915C068217930771F0F1
:10563000E0915906F0915A06E75EF94F4083909346
:105640005A068093590602C08091C600FF91EF91DF
:105650009F918F914F913F912F910F900FBE0F907F
:105660001F90189583EB95E00E94602A892B11F01A
:105670000E94F72A08951F920F920FB60F921124DD
:105680002F933F938F939F93EF93FF932091150652
:105690003091160680911706909118062817390741
:1056A00031F48091C1008F7D8093C10014C0E091DE
:1056B0001706F0911806EB52FA4F208180911706D9
:1056C0009091180601968F739927909318068093EE
:1056D00017062093C600FF91EF919F918F913F9104
:1056E0002F910F900FBE0F901F901895A0E0B0E083
:1056F000ECE7FBE20C94FF2CFC011382128288EE93
:1057000093E0A0E0B0E084839583A683B7838EE81E
:1057100093E0918380837587648757874687318BB1
:10572000208B138B028BF58AE48AD78AC68AB18EC6
:10573000A08E938E828E8F85848F8889858F8989AC
:10574000868F8A89878F8B8980A3ECE00C941B2D30
:10575000CF92DF92EF92FF92CF93DF93EC016A0139
:105760007B01411581EE580761057105F9F0EC895F
:10577000FD8981E090E008A002C0880F991F0A947B
:10578000E2F7808360E079E08DE390E0A701960185
:105790000E94B82C2150310941095109569547956D
:1057A00037952795211580E1380798F0EC89FD8918
:1057B000108260E874E88EE190E0A70196010E94F3
:1057C000B82C215031094109510956954795379513
:1057D0002795E889F9893083EA89FB89208319A212
:1057E000EE89FF89408181E090E09C010C8C02C031
:1057F000220F331F0A94E2F7422B4083EE89FF8980
:1058000040819C010D8C02C0220F331F0A94E2F7E5
:10581000422B4083EE89FF8940819C010E8C02C09F
:10582000220F331F0A94E2F7422B4083EE89FF894F
:1058300020810F8C02C0880F991F0A94E2F780958F
:1058400082238083DF91CF91FF90EF90DF90CF9004
:1058500008958F929F92AF92BF92CF92DF92EF9274
:10586000FF920F931F9381E08F9385E08F9387E0E2
:105870008F9383E08F9384E08F93E6EC8E2E912CB0
:10588000F2ECAF2EB12CA1ECCA2ED12CB0ECEB2E49
:10589000F12C04EC10E025EC30E045ED55E069E139
:1058A00076E083EB95E00E94762B0F900F900F909F
:1058B0000F900F901F910F91FF90EF90DF90CF907E
:1058C000BF90AF909F908F9008950E94A9270E944B
:1058D0000C21C2E3DBE20E94B0232097E1F30E9497
:1058E000322BF9CFA29FB001B39FC001A39F700DCF
:1058F000811D1124911DB29F700D811D1124911DD8
:1059000008950E94722CA59F900DB49F900DA49FA6
:10591000800D911D11240895B7FF0C94812C0E94D5
:10592000812C821B930B0895DB018F939F930E9420
:10593000812CBF91AF91A29F800D911DA39F900DCF
:10594000B29F900D1124089597FB072E16F4009432
:1059500007D077FD09D00E94362D07FC05D03EF414
:10596000909581959F4F0895709561957F4F08950B
:10597000A1E21A2EAA1BBB1BFD010DC0AA1FBB1F53
:10598000EE1FFF1FA217B307E407F50720F0A21BC5
:10599000B30BE40BF50B661F771F881F991F1A9432
:1059A00069F760957095809590959B01AC01BD015C
:1059B000CF010895052E97FB1EF400940E94F12C50
:1059C00057FD07D00E94B82C07FC03D04EF40C946E
:1059D000F12C50954095309521953F4F4F4F5F4F9B
:1059E000089590958095709561957F4F8F4F9F4F4B
:1059F00008952F923F924F925F926F927F928F9273
:105A00009F92AF92BF92CF92DF92EF92FF920F934D
:105A10001F93CF93DF93CDB7DEB7CA1BDB0B0FB657
:105A2000F894DEBF0FBECDBF09942A883988488814
:105A30005F846E847D848C849B84AA84B984C884AA
:105A4000DF80EE80FD800C811B81AA81B981CE0FA1
:105A5000D11D0FB6F894DEBF0FBECDBFED01089586
:105A6000EE0FFF1F0590F491E02D0994AA1BBB1BBC
:105A700051E107C0AA1FBB1FA617B70710F0A61B4E
:105A8000B70B881F991F5A95A9F780959095BC016F
:105A9000CD0108958F929F92AF92BF92CF92DF92E5
:105AA000EF92FF92CF93DF93EC01688179818A8135
:105AB0009B81611571058105910521F464E279ED01
:105AC0008BE597E02DE133EF41E050E00E94DA2CC6
:105AD00049015A019B01AC01A7EAB1E40E94812C63
:105AE0006B017C01ACEEB4EFA50194010E948F2CF8
:105AF000C60ED71EE81EF91EF7FE06C081E0C81AC2
:105B0000D108E10880E8F80AC882D982EA82FB82DB
:105B1000C701B6019F77DF91CF91FF90EF90DF90A3
:105B2000CF90BF90AF909F908F9008950E944A2D84
:105B3000089586E091E00E944A2D08956093060141
:105B400070930701809308019093090108952F92A3
:105B50003F925F926F927F928F929F92AF92BF928D
:105B6000CF92DF92EF92FF920F931F93CF93DF9329
:105B70008B01EA016115710521F0DB018C9311960F
:105B80009C93209739F09E01225031092332310530
:105B900008F0D8C07C016701BFEFCB1ADB0A5601C1
:105BA000F7016080862D90E00E94D92E892B11F09C
:105BB0007601F1CFFDE26F120AC0570182E0A80E14
:105BC000B11CD70111966C90772473940BC0BBE283
:105BD0006B1207C05701E2E0AE0EB11CD70111965F
:105BE0006C90712CCE018F7E892B89F4B0E36B12FF
:105BF00037C0F50180818F7D8835D1F46180F2E076
:105C0000AF0EB11C872D8260782EC0E1D0E0CA3083
:105C1000D10551F1C031D10521F0C830D10599F439
:105C200009C0CC24CA94DC2CEC2CAFE0FA2E22C0A4
:105C3000209769F7C8E0D0E0CC24CA94DC2CEC2C87
:105C4000FFE1FF2E17C06FEF7FEFCB019E014427CE
:105C500037FD4095542F0E94B82C69017A010AC083
:105C60002097A9F6CAE0D0E0E9E9CE2EDC2CEC2C96
:105C7000E9E1FE2EF50160E020E030E0A9014E01EF
:105C8000AA2497FCA094BA2C1F0170ED572E560C35
:105C9000A9E0A51570F48FEB860D8A3118F499EC04
:105CA000592E06C08FE9860D8A3148F589EA582EAB
:105CB000560C852D90E08C179D070CF56F3FD9F0A1
:105CC000C216D306E406F50698F0C501B4010E9499
:105CD000942C9B01AC01852D90E0A0E0B0E0280F52
:105CE000391F4A1F5B1F281739074A075B0710F443
:105CF0006FEF01C061E03196D1016C90C5CF011505
:105D0000110551F0662311F0319703C071FE04C0F4
:105D10003297D801ED93FC9370FE07C050954095E3
:105D2000309521953F4F4F4F5F4F67FF10C082E284
:105D300090E090935E0680935D066FEF7FEF8FEFAC
:105D40009FEF07C060E070E080E090E002C0B90122
:105D5000CA01DF91CF911F910F91FF90EF90DF90DB
:105D6000CF90BF90AF909F908F907F906F905F90FB
:105D70003F902F900895FC0188279927E89421915E
:105D80002032E9F3293010F02E30C8F32B3241F0E5
:105D90002D3239F4689404C00E940D2F820F911D9A
:105DA000219120532A30C0F31EF4909581959F4F86
:105DB0000895911150C0803219F089508550D0F764
:105DC00008954AE953E00E94E62E0895FA01A19150
:105DD000B081009719F41097E1F0CD01DC01CD01FD
:105DE0000D90002011F4C00113C0FB01219122236A
:105DF00019F02015D9F7F3CFFB012191201519F4E3
:105E00001E92119606C02223C1F70D900020A1F723
:105E1000D001FA01A193B08308957AE0979F902D65
:105E2000879F802D910D11240895F999FECF92BD81
:105E300081BDF89A992780B50895262FF999FECF4C
:105E40001FBA92BD81BD20BD0FB6F894FA9AF99A97
:105E50000FBE01960895992788270895F894FFCFDB
:105E600000005F06200001000000FF0002000200A9
:105E70000200020002000200020002000200020012
:105E8000020002000200020002000280250000055C
:105E9000400AA1204EA50020244EA52C2330C0127C
:105EA00000001A400AA1204EA5001B1E27522C23D9
:105EB000308025000005400AA1204EA50020244E78
:105EC000A52C2330004B000006400AD0009D49005D
:105ED0007B289D492C233000E1000005400A450144
:105EE000D7DC03B81E0EBF00232E48E801008A400D
:105EF0000A6001555502AD1E20000023C801545808
:105F00002074696D656F75742100596573004E6F5B
:105F1000002C00386368004E2F41002C205B005D90
:105F20002028002900486F70206368616E6E656CE0
:105F30002000204020007363616E6E6572206D6FDB
:105F40006465004E4F5420454E41424C4544005339
:105F5000656E64696E672073657474696E6773201B
:105F6000746F2052580A00526573657474696E67C5
:105F70002073657474696E6773206F6E2052580ABF
:105F80000041626F727465642065646974730A000D
:105F9000696E76616C69642073656C656374696FA2
:105FA0006E000D0A496E76616C696420696E7075C9
:105FB00074202D2064697363617264656421070035
:105FC00053657474696E67732073617665642074B9
:105FD0006F20454550524F4D0A00526576657274E8
:105FE00065642073657474696E67732066726F6D83
:105FF00020454550524F4D0A004C6F616465642046
:10600000666163746F72792064656661756C747320
:106010000A004B657920616E64206368616E6E656D
:106020006C732072616E646F6D697A65640A004FEB
:1060300070656E4C52536E672054582073746172B1
:1060400074696E672000206F6E20485720006D6FC6
:1060500064756C65206C6F636B65643F00342B3432
:10606000003800382B340031320031322B3400310B
:10607000360050504D005253534900534441005391
:10608000434C00525844005458440041494E004C7F
:10609000424545500053504B54524D0053425553C6
:1060A0000053554D44004C4C494E440000070B0C26
:1060B00010111500B701FD020103030307030A03D2
:1060C0000F03B701160A13223129120316031B030B
:1060D0001F03230327032B032F0335033C03410333
:1060E00046035F025F025F025F0200000000BA2AFF
:0A60F000BF28602A8D2A722AAF2A09
:00000001FF
